:02000004F90001
:1000000097110000938181AC23A00182732540F1F8
:1000100015C503A5018275DD0F0020020F10000039
:1000200083A7C181014581450146828723AEA18016
:100030000F001001054523A0A182828013818192C7
:1000400013850181938501811386C18163FAC500FF
:100050008322050023A0550011059105E3EAC5FEA2
:100060001385C181938581826377B50023200500C4
:0E0070001105E36DB5FEDD2A192001A0828086
:10007E00B70701E81307E01098C7B70701E81D4757
:10008E00D8C771A8B70603E8416791067D179C4251
:10009E00F98FF5DF856793870780370703E81CC361
:1000AE008280B70603E8416791067D179C42F98F5F
:1000BE00F5DF13070020B70703E898C3370703E8F7
:1000CE0011071C43C183F5DFB70703E88843137597
:1000DE00F50F8280B70603E8416791067D179C42B3
:1000EE00F98FF5DF13650510B70703E888C3828023
:1000FE00B7C7B0F8E11794439386A60F984333879A
:10010E00E640E35D07FEB70603E8416791067D17FB
:10011E00130600109C42F98FE39EC7FE82804111A8
:10012E0006C622C426C2B70703E823A40700094760
:10013E00B70703E898D39546B70703E8D4D3B707B4
:10014E0003E898D71D47B70703E8D8D755371D3FA3
:10015E00B70603E8416791067D179C42F98FF5DFDC
:10016E00856793870788370703E81CC31305B00A12
:10017E009537093FB53FB7C7B0F8E11794431967F4
:10018E001307871ABA9698433387E640E35D07FE56
:10019E00B70603E8416791067D179C42F98FF5DF9C
:1001AE00856793870788370703E81CC31305F00993
:1001BE001537C53DB7C7B0F8E11794434967130724
:1001CE00874F2A84BA9698433387E640E35D07FE4D
:1001DE00553D393FB70603E8416791067D179C42AE
:1001EE00F98FF5DF856793870788370703E81CC308
:1001FE009307D009130590026304F4001305900EC3
:10020E00D13D4935F535B70603E8416791067D17AF
:10021E009C42F98FF5DF856793870788370703E8D8
:10022E001CC32D45453D130500046D3501455D3557
:10023E0001454D350145793D0564B70402009535FC
:10024E00A2872380A7000504E31B94FE253D0565C8
:10025E00F9332244B24092448567410182874111AD
:10026E0022C44AC097070000938747061704000070
:10027E001304C40506C626C233898740638B8700E4
:10028E001359294081441C40850411048297E3ECE4
:10029E0024FF9707000093876703170400001304D9
:1002AE00E4023389874013592940638987008144CA
:1002BE001C40850411048297E3EC24FFB2402244D3
:0802CE009244024941018280C3
:0C02D6000000000000000000000000001C
:04000005F9000000FE
:00000001FF
